:107800000C942A3C0C94453C0C94453C0C94453C0F
:107810000C94453C0C94453C0C94453C0C94453CE4
:107820000C94453C0C94453C0C94453C0C94453CD4
:107830000C94453C0C94453C0C94453C0C94453CC4
:107840000C94453C0C94453C0C94453C0C94453CB4
:107850000C94453C11241FBECFE5D8E0DEBFCDBF60
:1078600010E0A0E6B0E0ECE1FFE702C005900D9269
:10787000A436B107D9F711E0A4E6B0E001C01D922B
:10788000A63AB107E1F70C94513F0C94003C0F92DB
:10789000AF93BF93CF93DF93EF93FF93FC01EA0184
:1078A000DB01C895099231961197D9F7FF91EF91B5
:1078B000DF91CF91BF91AF910F9008950F921F92DA
:1078C0000F93AF93BF93CF93DF93EF93FF93FC019D
:1078D000EA01DB010990199001E043D0329612973A
:1078E000C9F7FC0103E03DD005E03BD0FF91EF91EB
:1078F000DF91CF91BF91AF910F911F900F9008959D
:107900000F931F93EF93FF93FC0103E02AD000E84D
:1079100010E0E00FF11FE617F707B9F7FF91EF91BD
:107920001F910F9108950F930F9222D0082E09E016
:1079300018D00F900F9108950F930F92EF93FF932C
:1079400017D0FC0160935700C895802DFF91EF91EF
:107950000F900F9108950F930BD001E102D00F917A
:107960000895E199FECF00935700E895FFFF0000CE
:107970000091570000FDFCCF089589E089B98AB1D4
:1079800088618AB908958AB1877E8AB908958CB9C9
:107990005E9BFECF5E9A08958CB1992708958BB1B6
:1079A0009927807890700895EF92FF920F931F931C
:1079B000CF93DF937B01C0E0D0E0C617D70770F408
:1079C0008C010E94CF3C8823E1F30E94CC3CF8015B
:1079D00081938F012196CE15DF0598F381E090E029
:1079E000DF91CF911F910F91FF90EF900895EF924B
:1079F000FF920F931F93CF93DF937C018B01C0E025
:107A0000D0E0C017D10738F4F70181917F010E94BF
:107A1000C73C2196F6CF81E090E0DF91CF911F9196
:107A20000F91FF90EF900895EF92FF920F931F93A5
:107A3000CF93DF937C0100E010E00817190788F46A
:107A4000C0E0D0E000000E94CF3C882351F4219692
:107A500088E0CA3CD807B0F30F5F1F4F0E151F0513
:107A600078F3DF91CF911F910F91FF90EF900895E0
:107A70000E94C33C0E9400000895DF92EF92FF92A3
:107A80000F931F93CF93DF93CDB7DEB72197DEBF60
:107A9000CDBF8C017B011982D98061E070E0CE01FD
:107AA000860F971F0E94D43C89818B31B1F761E02A
:107AB00070E0C8010E94D43C61E070E0CE01860F06
:107AC000971F0E94D43C89819927182F002761E0D5
:107AD00070E0CE01860F971F0E94D43C8981080F69
:107AE000111D61E070E0CE01860F971F0E94D43C0B
:107AF00089818E30B9F4C8010196BC01C7010E948A
:107B0000D43C98018FEF0F3F180779F0F70181916E
:107B10007F01D82621503040FFEF2F3F3F07B1F7BC
:107B2000DD2019F080E090E001C0C8012196DEBFA1
:107B3000CDBFDF91CF911F910F91FF90EF90DF901C
:107B40000895CF92DF92FF920F931F93CF93DF930D
:107B5000182FEB016A018BE10E94C73C4BE1F42E28
:107B6000812F0E94C73CF1260D2F1127802F0E94E4
:107B7000C73CF0268C2F0E94C73CFC268EE00E945A
:107B8000C73C8EE0F82621978FEFCF3FD80759F0FA
:107B9000F60181916F01F8260E94C73C2197FFEF03
:107BA000CF3FDF07A9F78F2D0E94C73CDF91CF9110
:107BB0001F910F91FF90DF90CF9008959927813901
:107BC000910559F08239910524F48039910529F005
:107BD00008C08239910519F004C082E003C087E033
:107BE00001C080EC99270895BF92CF92DF92EF9267
:107BF000FF920F931F93CF93DF93B82E8B01FB015E
:107C00008081C82FDD27C231D10509F46DC0C33191
:107C1000D105DCF4C330D10509F44DC0C430D10521
:107C200044F4C130D10579F1C230D10509F44AC01C
:107C300004C1C630D10509F44AC0C630D1050CF4E0
:107C4000FCC060970CF4F9C055C0C531D10509F4EA
:107C5000C8C0C631D10544F4C331D10509F472C09E
:107C6000649709F44AC0E9C0CA31D10509F4D7C004
:107C7000CB31D10524F4669709F49AC0DEC06B9726
:107C800009F4C4C0DAC0FB01118288E0828381E478
:107C9000838386E5848382E5858389E4868383E51F
:107CA000878380E580878FE5818782E38287AB01C8
:107CB0006BE070E0C8C0FB0181810E94DE3DF801ED
:107CC000828301C0FB011182A801BE01BCC0FB017F
:107CD00083819927982F88272481820F911D909363
:107CE000A5018093A40107C060E070E880E090E007
:107CF0000E94803CF8011182A3C0FB018181992779
:107D0000D82FCC2782819927C82BD92B1182CB0160
:107D100002962091A4013091A501AC01BE01C901D8
:107D2000880F991F0E94473CF801EC0FFD1F12823B
:107D30009E01369527958091A4019091A501820F0F
:107D4000931F49C0FB0181819927D82FCC278281BD
:107D50009927C82BD92BCC24DD24CC16DD06D8F4EA
:107D6000FAE0EF2EF12CE60EF71E8091A40190911F
:107D7000A501880F991FA70160E870E08C0D9D1D7B
:107D80000E945E3C80E890E0C80ED91EE80EF91E05
:107D9000CC16DD0650F30E94AB3CF8011182D6955B
:107DA000C7958091A4019091A5018C0F9D1F29C0BA
:107DB000FB0181819927D82FCC2782819927C82B55
:107DC000D92B1182EC0FFD1F12828091A40190919A
:107DD000A5018C0F9D1F9093A5018093A40123966C
:107DE00073CFFB0181819927382F22278281992720
:107DF000282B392B11828091A4019091A501820F2B
:107E0000931F9093A5018093A4011AC0FB011182D6
:107E10008481E82FFF27E05AFF4F808107C0FB01D4
:107E2000118269E081E090E00E949C3CF80182832D
:107E30001382A80164E070E006C089ECF801818338
:107E4000A80162E070E08B2D0E94A13DDF91CF91EF
:107E50001F910F91FF90EF90DF90CF90BF9008950A
:107E6000CF93DF93CDB7DEB72197DEBFCDBF69E0FB
:107E700081E090E00E949C3C992784FF09C08F7E9E
:107E80000E94933C05C064E670E089810E94F43D45
:107E900064E670E0CE0101960E943D3D892B99F386
:107EA000F7CFCFE5D8E0DEBFCDBFCEE1F894AEEF9F
:107EB000B3E00E94853F802D843B71F4AFEFB3E0C7
:107EC0000E94853F802D833C39F4ADEFB3E00E94E2
:107ED000853F802D992781BF0E94BD3C0E94CC3CEC
:107EE00084E690E00E94143D0E94CF3C882319F064
:107EF0000E94303F04C0C150C8BBCC2389F70E9408
:107F0000383D80E090E00C948D3FE199FECFBFBBFF
:0C7F1000AEBBE09A11960DB20895FFCFB1
:047F1C001E950200AC
:040000030000780081
:00000001FF
